:100000008BC0A3C0A2C0A1C0A0C09FC09EC09DC005
:100010009CC09BC09AC099C098C097C096C0000071
:1000200000000000000000000000000000000000D0
:1000300000000000000000000000000205080B0E98
:1000400012161A1E22272C31363B41474D545B6253
:100050006971798189929BA4AEB8C2CDD8FF0303A0
:10006000040506080A0C0F13171C21282F373F49D7
:10007000545F6C7A8999ABBED2E8FFFFFFFFFFFFA8
:10008000FFFFFFFFFFFFFFFFFFFFFFFFFFFFFFFF80
:10009000FFFFFFFFFFFFFFFFFFFFFFFFFF0040002D
:1000A0000000000000000B400000000000000B23D7
:1000B0004000000000000B1A2E40000000000B174B
:1000C0002432400000000B141F29354000001D4061
:1000D000F80000000000FAFE0B1D400000000912AD
:1000E0001D2E400000000B1D3200FAFEF8405F4557
:1000F000644669476F48744979607E6183628963A9
:100100008E64936598669E67A368A869AD80B28186
:10011000B882BD83C284FF2111241FBECFEDCDBFA5
:1001200010E0A0E6B0E0E0E7F7E002C005900D9235
:10013000A636B107D9F720E0A6E6B0E001C01D92CF
:10014000AC37B207E1F776D111C35ACF815090E0B6
:10015000FC01E25AFF4F2491FC01E25EFF4F8491C3
:1001600088BD29BD089520ED37E0019720F0F90101
:100170003197F1F7FACF089588EE93E0F4CF369AED
:100180003699FECF85B10895CF93C091660081E086
:100190008C0F8F73809366006091670090E0D8D2D7
:1001A0006FEF8C2F90E0CF91D3C2609163008EE708
:1001B00090E0CED260916A008DE790E0C9D2609164
:1001C00061008CE790E0C4D2609160008BE790E022
:1001D000BFD2609168008AE790E0BAD26091620075
:1001E00089E790E0B5D260916B0088E790E0B0D2EB
:1001F0006091690087E790E0ABD2609164008FE77F
:1002000090E0A6D2C1CFCF938FE790E099D2853509
:1002100011F0CF91CACF10926600C0916600C03431
:1002200060F48C2F90E08CD28F3F19F080936700A0
:1002300004C0CF5FC0936600F0CF8EE790E080D21D
:10024000809363008DE790E07BD280936A008CE717
:1002500090E076D2809361008BE790E071D280933A
:1002600060008AE790E06CD28093680089E790E0B4
:1002700067D28093620088E790E062D280936B003F
:1002800087E790E05DD280936900CF910895209137
:1002900063009091620040916B0080916900882317
:1002A00019F040E090E029E030E083E0220F331FB6
:1002B0008A95E1F7F901E256FF4F992331F081E089
:1002C00080936E00AFE6B0E002C0AEE6B0E080E042
:1002D000883029F480936D00EAEEF0E008C0549174
:1002E0005523C1F354915D938F5F3196F1CF5491B3
:1002F0005D93319650E0EE3EF507C8F354E0580F99
:1003000050937B004423F1F0482F50E0FA01E20FB4
:10031000F31FE256FF4FAEE6B0E0BD012A2F261BC9
:10032000022E000C330B2417350724F43197249147
:100330002D93F4CF992311F021E02C9323E0280F83
:1003400020937B00992341F090917B009F5F9093D5
:100350007B008F5F80936D000895811103C018BCEE
:1003600019BC0895F3CECF93DF93D82F90916C00F2
:100370002D2F291BC1E009F4C0E025952595C22B3E
:10038000C90FC0936C008C2FE8DF80E190E0EBDEBA
:10039000DC13ECCFDF91CF9108950F931F93CF9390
:1003A000C82F8B01CC2361F080E1D0DEC801DBDEF9
:1003B00018BC19BCC801D7DEC801D5DEC150F2CFC8
:1003C000CF911F910F9108951F93CF93DF93EC016D
:1003D000862F6EE370E0E1DF888111E0812788835A
:1003E000E4DE6FE070E080E2D8DF888118271883B0
:1003F000DCDEDF91CF911F91BFCE1F93CF93DF93B0
:100400008FEA87B986EC86B9BADE10E1C0E0D0E0A9
:10041000B6DEC80FD11D85E090E0A5DE1150C1F712
:10042000CE0124E0969587952A95E1F7DF91CF914B
:100430001F910895A39A83EA87B986EC86B9369905
:10044000FECF369A3699FECFC5B1B99AB89A81EAED
:100450008ABD81E083BFD7DE1ADF809168008111F9
:100460003AC0CF3B90F080917C008F5F8F7180937A
:100470007C00809167008F5F8093670090916D0092
:10048000891748F11092670026C010927C00CF3582
:10049000D0F0209161008091670090916D0022233F
:1004A00021F020916900222321F08F5F8093670063
:1004B000E7CF891739F3811102C080917B00815009
:1004C0008093670008C0809169008111DBCF809123
:1004D0006A008823B9F258DEBB9AC39AA29A81EACD
:1004E00087B986EC86B9369AD0916700ED2FF0E097
:1004F000E259FF4FC08180916800882319F0109263
:100500007C0001C0DC2FF12C10E081EAD82E96ECA3
:10051000C92EEE24EA942DEFB22E3CEFA32E80914B
:100520007C008031C8F128DE10927C0010926700B8
:1005300061E089E690E048DF809169008111EFCFAA
:1005400062E08AE690E040DF63E082E690E03CDF34
:1005500064E08BE690E038DFB092670065E088E603
:1005600090E032DF1092670066E081E690E02CDFD9
:10057000A092670067E088E690E026DF10926700AF
:1005800068E084E690E020DFE0916700F0E0E25967
:10059000FF4FD081CD2FA7C0D83FD9F408E080E429
:1005A000D5DD84E190E0DFDD18BC19BC88E290E085
:1005B000DADD0150A1F708E080E4C8DD88E290E0D0
:1005C000D2DD18BC19BC80E590E0CDDD0150A1F76B
:1005D0008AC0DA3F81F404E0E8BC19BC85E090E011
:1005E000C2DD18BCE9BC81E490E0BDDD0150A1F79B
:1005F00080ED92E077C0DE3F51F584E690E0B3DD18
:10060000BEDD90E0292F30E0F901E251FF4FE49187
:10061000E81710F49E5FF6CFF901E151FF4F049106
:100620006EE370E0802F829586958770B6DE84EF4A
:1006300091E099DD65E070E081E0AFDE8EEE92E062
:1006400092DD6EE370E0802F8F71A7DE11C0DD3F79
:1006500091F4109267001092680000E0009363002C
:10066000A4DD66EA70E081E098DE0F5F0930B1F743
:1006700083DD82DD38C0DC3FA9F410926700109260
:1006800068008FEF8093600090DD80E16CDE74DDA8
:1006900073DD80E468DEB1DE8093600086DD6CDDB2
:1006A0006BDDF9CF8C2F5FDEA8DE20916000821712
:1006B00038F01F5F103178F0C93068F0C1500AC0BF
:1006C00090E030E022503109821793071CF4CD17D7
:1006D00008F4CF5F10E08C2F46DEA29AD7B8C6B8D8
:1006E00084EF91E040DD10927C00349B18CF85B1FF
:1006F000893718F5F39487E08F1500F5C134C0F4FD
:10070000C23038F08C2F86958695C695DC2FD80F91
:1007100010C018BC19BC85B7877E806185BF85B7BE
:10072000806285BF889585B78F7D85BFDC2F01C02E
:10073000D0E28D2F18DE20DDCD2FF12C369AEFCEB2
:10074000E199FECF1FBA8EBBE09A99278DB3089529
:10075000262FE199FECF1CBA1FBA8EBB2DBB0FB658
:10076000F894E29AE19A0FBE01960895F894FFCFAB
:060770004F0101055500D8
:00000001FF
